:100000000C9417060C942F290C945C290C943F0631
:100010000C943F060C943F060C943F060C943F064C
:100020000C943F060C943F060C94C50C0C943F06B0
:100030000C943F060C943F060C943F060C943F062C
:100040000C9489290C943F060C94432D0C947E2D1E
:100050000C943F060C943F060C943F060C943F060C
:100060000C943F060C943F06591C601C601C591CE4
:10007000601C601C601C601C601C601C601C601CA0
:10008000601C601C601C601C601CCE1B601C601C23
:10009000601C601C601C381B601C601C601C601CA9
:1000A000601C601C601C601C601C601C601C601C70
:1000B000601C601C601CDA1BDA1BDA1BDA1BDA1B03
:1000C000DA1BDA1BDA1BDA1B601C601C601C601C6C
:1000D000601C601C381BD91BD91BD91BD91B601C89
:1000E000EA1BF21BFA1B021C0A1C121C1A1C221C03
:1000F0002C1C361C401C4A1C7D1B3D1B601C601CBC
:10010000601C601CCE1B601C601C601C601C601CA2
:10011000601C601C601CD81BD81BD81BD81B601C23
:10012000EA1BF21BFA1B021C0A1C121C1A1C221CC2
:100130002C1C361C401C4A1C7D1B3D1B601C601C7B
:10014000601C601CCE1B911C911C911C911C911C6D
:10015000911C911C911C911C911C911C911C911C37
:10016000B11DB11DB11DB11DB11DB11DD81CE21CC9
:10017000EC1CF61C5C1D661D741D851D221E921E46
:10018000631E681E6D1E721E771E7C1E811E921ECF
:100190008C1EAB25C025CC25D525E22508261026AA
:1001A00033262026456E746572206D656E752E2E81
:1001B0002E00546F67676C6564206D6963726F50C1
:1001C000504D00546F67676C656420696E76657288
:1001D0007465642050504D2100546F67676C6564EE
:1001E000205458206D7574696E672100546F6767DD
:1001F0006C65642074656C656D657472792100505E
:10020000726F746F636F6C206572726F72207769A2
:1002100074682052580054696D656F757420776852
:10022000656E20636F6E6E656374696E6720746FB0
:1002300020525800507265737320616E79206B658F
:100240007920746F2063616E63656C00436F6E6E1E
:10025000656374696E6720746F2052582C20706F2C
:100260007765722075702074686520525820287751
:100270006974682062696E6420706C7567206966B5
:10028000206E6F74207573696E6720616C77617979
:10029000732062696E642900546F67676C6564201F
:1002A00027696D6D656469617465206F757470751B
:1002B000742700546F67676C65642027736C6176E0
:1002C00065206D6F64652700546F67676C656420F7
:1002D00027616C776179732062696E642700546FBF
:1002E00067676C65642050504D206368616E6E6571
:1002F0006C206C696D6974005365742052535349C6
:1003000020696E6A656374696F6E206368616E6EE2
:10031000656C2028303D3D64697361626C6529001D
:100320005365742050504D206D696E696D756D2058
:1003300073796E630053657420626561636F6E202C
:10034000696E74657276616C0053657420626561D4
:10035000636F6E2064656C6179005365742062651B
:1003600061636F6E206672657175656E6379206971
:100370006E20487A3A20303D64697361626C652C66
:100380002050783D504D52206368616E6E656C2040
:10039000782C2046783D465253206368616E6E6526
:1003A0006C2078005365742050574D2073746F7023
:1003B0002064656C61792028302064697361626C07
:1003C00065642C20312D323535203D3D20302E31D5
:1003D00073202D2035306D696E29005365742050CF
:1003E000504D2073746F702064656C6179202830E3
:1003F0002064697361626C65642C20312D3235355F
:10040000203D3D20302E3173202D2035306D696E1A
:100410002900536574206661696C736166652064A8
:10042000656C61792028302064697361626C656451
:100430002C20312D323535203D3D20302E3173209A
:100440002D2035306D696E29002A2A2A2A2A2A2A67
:100450002A2A2A2A2A2A2A2A2A2A2A2A2A2A2A2AFC
:100460002A2A2A2A2A2A0052582041636B656420CE
:100470002D2072657665727420737563636573737E
:1004800066756C21002A2A2A2A2A2A2A2A2A2A2A36
:100490002A2A2A2A2A2A2A2A2A2A2A2A2A2A2A2ABC
:1004A0002A2A002A2A2A2A2A2A2A2A2A2A2A2A2AD6
:1004B0002A2A2A2A2A2A2A2A2A2A2A2A2A2A2A2A9C
:1004C0000052582041636B6564202D207570646173
:1004D0007465207375636365737366756C21002A98
:1004E0002A2A2A2A2A2A2A2A2A2A2A2A2A2A2A2A6C
:1004F0002A2A2A2A2A2A2A2A2A2A2A2A0056616CE1
:1005000069642063686F69636573206172653A206E
:100510005B315D2D5B31365D20286368616E6E65F1
:100520006C20312D31362900536574206F7574703D
:10053000757420666F7220706F727420005B585D56
:100540002061626F7274206368616E6765732061F9
:100550006E64206578697420525820636F6E6669F6
:1005600067005B535D207361766520736574746901
:100570006E677320746F205258005B525D20726565
:10058000766572742052582073657474696E67734F
:1005900020746F2064656661756C747300557365B3
:1005A000206E756D62657273205B312D445D207421
:1005B0006F206564697420706F727473205B452DC1
:1005C000515D20666F722073657474696E67730085
:1005D000202D20726563656976657220636F6E6693
:1005E0006967757261746F722C207278207377203E
:1005F000000A0A6F70656E4C52536E672000536597
:10060000742073657269616C2062617564726174D3
:10061000653A200056616C69642063686F696365A0
:10062000733A2031202D20342B34202F2032202DDE
:100630002038202F2033202D20382B34202F203419
:10064000202D203132202F2035202D2031322B3407
:10065000202F2036202D203136005365742043682A
:10066000616E6E656C20636F6E6669673A20005339
:1006700065742044617461726174652028302D3284
:10068000293A200053657420486F70206368616EBA
:100690006E656C7320286D61782032342C20736570
:1006A0007061726174656420627920636F6D6D6141
:1006B00073292076616C69642076616C756573209E
:1006C000312D3235353A2000536574206368616EF0
:1006D0006E656C2073706163696E672028783130B5
:1006E0006B487A293A200053657420524620706F77
:1006F0007765722028302D37293A20005365742001
:100700005246206D616769632028686578292065F5
:100710002E672E20307844454144463030443A20FC
:10072000005365742062617365206672657175653A
:100730006E63792028696E20487A293A20005B5A36
:100740005D20656E74657220726563656976657299
:1007500020636F6E66696775726174696F6E20756C
:1007600074696C79005B465D20646973706C6179B3
:100770002061637475616C206672657175656E6366
:100780006965732075736564005B525D2063616CFD
:1007900063756C6174652072616E646F6D206B654A
:1007A0007920616E6420686F70206C697374005BDF
:1007B000495D207265696E697469616C697A65204A
:1007C00073657474696E677320746F20736B6574DE
:1007D00063682064656661756C7473005B585D20A6
:1007E000726576657274206368616E6765732061F7
:1007F0006E642065786974206D656E75005B535D6D
:1008000020736176652073657474696E67732074F4
:100810006F20454550524F4D20616E6420657869C8
:1008200074206D656E7500557365206E756D62651B
:100830007273205B302D395D20746F20656469749C
:1008400020706172616D657465727300202D205394
:10085000797374656D20636F6E6669677572617414
:10086000696F6E000A0A6F70656E4C52536E672096
:10087000005129204F7574707574206265666F721F
:1008800065206C696E6B20283D465329203A200074
:10089000502920536C617665206D6F646520286552
:1008A00078706572696D656E74616C293A20004FCD
:1008B000292054696D65642042494E4420617420AA
:1008C0007374617274757020203A20004E29205094
:1008D000504D206F7574707574206C696D69746506
:1008E0006420202020203A200044495341424C45B6
:1008F00044004D292050504D205253534920746FCD
:10090000206368616E6E656C202020203A20004CC8
:10091000292050504D206D696E696D756D20737979
:100920006E63202875732920203A200044495341E2
:10093000424C4544004B29204661696C73616665F1
:1009400020626561636F6E20696E74762E20283197
:100950002D32353573293A20004A29204661696CC9
:100960007361666520626561636F6E2064656C61AA
:10097000792028302D323535203D3E20313073200E
:100980002D203135306D696E293A200049292046E5
:1009900061696C7361666520626561636F6E206674
:1009A00072712E203A200048292050574D20737430
:1009B0006F702064656C6179202020202020203A0F
:1009C000200047292050504D2073746F70206465BB
:1009D0006C6179202020202020203A200046292008
:1009E0004661696C736166652064656C617920207D
:1009F00020202020203A200050574D206368616E4F
:100A00006E656C200066756E6374696F6E3A2000C7
:100A10002920706F72742000506F776572546F7761
:100A2000657200445446205548462033322D626991
:100A3000742031306368004F70656E4C52536E679E
:100A40005258206D696E6920342F36636800466CF9
:100A50007974726F6E2F4F72616E676552582055B0
:100A600048462038636800525820747970653A20EF
:100A70000044697361626C656400487A00203D3D02
:100A8000200043616C63756C617465642070616300
:100A90006B657420696E74657276616C3A200042F1
:100AA00029204D6963726F202868616C6629205087
:100AB000504D202020203A00412920496E76657251
:100AC0007465642050504D20696E20202020203A0B
:100AD000003029204D7574652062757A7A65722020
:100AE000286D6F73746C79293A0039292053657227
:100AF00069616C2062617564726174653A00736D3E
:100B0000617274506F7274004672536B7900547244
:100B1000616E73706172656E740044697361626CBA
:100B200065640038292054656C656D657472793A86
:100B300020202020202020003729204368616E6E6D
:100B4000656C20636F6E6669673A20200036292045
:100B500044617461726174652028302D32293A2015
:100B6000202000352920486F70206368616E6E6513
:100B70006C733A2020202020003429204368616EC5
:100B80006E656C2073706163696E673A2020003374
:100B90002920524620706F7765722028302D372922
:100BA0003A202020003229205246206D6167696377
:100BB0003A202020202020202020003129204261BE
:100BC0007365206672657175656E63793A202020C1
:100BD0000000000000240027002A0000000000257B
:100BE0000028002B0000000000230026002900043C
:100BF00004040404040404020202020202030303C4
:100C000003030301020408102040800102040810BD
:100C1000200102040810200000000700020100006B
:100C2000030406000000000000000000262F11242D
:100C30001FBECFEFD8E0DEBFCDBF13E0A0E0B1E034
:100C4000EEE8F0E602C005900D92A839B107D9F799
:100C500016E0A8E9B3E001C01D92AD35B107E1F798
:100C60001CE0CEE2DCE004C02297FE010E942230AC
:100C7000CC32D107C9F70E946B2F0C9445300C94ED
:100C80000000A0E0B0E0E7E4F6E00C94F12FEC0106
:100C9000A880B980CA80DB80A114B104C104D1044A
:100CA00041F484E2A82E89EDB82E8BE5C82E87E0AA
:100CB000D82EC601B5012DE133EF41E050E00E948E
:100CC000CE2F27EA31E440E050E00E947A2F7B01EA
:100CD0008C01C601B5012DE133EF41E050E00E94E7
:100CE000CE2FCA01B9012CEE34EF4FEF5FEF0E9417
:100CF0007A2F6E0D7F1D801F911F97FF04C06150DA
:100D0000704080409048688379838A839B839B01ED
:100D1000AC015F77B901CA01CDB7DEB7EAE00C9448
:100D20000D300E944106089581EB92E00E94410639
:100D300008956093B1027093B2028093B3029093CE
:100D4000B4020895A0E0B0E0E8EAF6E00C94EA2FDF
:100D5000EC012B016A016115710519F0FB0191830A
:100D60008083C114D10449F0C6010297839728F00B
:100D700020E030E040E050E0DCC0A9908A2D90E017
:100D80000E943A30892BC9F7FDE2AF1621F4A990F1
:100D90003324339405C08BE2A81609F4A9903324B8
:100DA000C114D10421F0E0E1CE16D10411F5F0E335
:100DB000AF1669F48881883711F0883541F4A9802D
:100DC000229682E0382A20E1C22ED12C12C0C11412
:100DD000D10479F4E0E3AE1659F199E9E92E99E9E5
:100DE000F92E99E9092F99E1192F8AE0C82ED12C03
:100DF0003AC0FAE0CF16D10491F080E1C816D104D0
:100E000029F0E8E0CE16D104F9F415C0BFEFEB2EBF
:100E1000BFEFFB2EBFEF0B2FBFE01B2F24C0A9E9B4
:100E2000EA2EA9E9FA2EA9E90A2FA9E11A2F1BC077
:100E3000F8E0CF2ED12CEFEFEE2EEFEFFE2EEFEFFE
:100E40000E2FEFE11E2F0FC09601442737FD40956E
:100E5000542F6FEF7FEF8FEF9FEF0E94AC2FC901F0
:100E6000DA017C018D0120E030E040E050E060E0FC
:100E70003601882477FC8094982C70EDB72EBA0C3C
:100E8000F9E0FB1570F48A2D81548A3118F499EC3D
:100E9000B92E06C08A2D81568A3148F589EAB82EC6
:100EA000BA0C8B2D90E08C159D050CF56F3FE9F089
:100EB000E216F30604071507B8F0CA01B901A40148
:100EC00093010E947A2F9B01AC018B2D90E0A0E052
:100ED000B0E0280F391F4A1F5B1F281739074A0740
:100EE0005B0710F061E001C06FEFA990C6CF41141D
:100EF000510451F0662311F0219703C031FE04C064
:100F00002297F201D183C08330FE07C050954095EF
:100F1000309521953F4F4F4F5F4F67FF0AC082E2E8
:100F200090E090935C0680935B062FEF3FEF4FEFCE
:100F30005FEFB901CA01CDB7DEB7E1E10C9406302D
:100F4000FC0188279927E89421912032E9F3293080
:100F500010F02E30C8F32B3241F02D3239F4689462
:100F600004C00E94F507820F911D219120532A3061
:100F7000C0F31EF4909581959F4F089548E953E082
:100F80000E94C3070895009731F4DA018D919C9176
:100F9000009709F40EC0DC01FB013D912191222351
:100FA00019F03217C9F3FACF332331F4DA011D9265
:100FB0001C928827992708951197AF93BF93FB013F
:100FC0003D912191321771F4332321F48827992719
:100FD000119702C01E921196FA01A193B0839F91BE
:100FE0008F910895222369F7EACF7AE0979F902D99
:100FF000879F802D910D1124089580919A0381304F
:1010000019F482E080939A0380919A03833019F453
:1010100084E080939A030895E3E0F0E089E0809310
:101020005700849190E08670863009F491E0892F12
:1010300008951F93182F0E940C08882379F09FB7FA
:1010400081E08093A305F894A89588E180936000DF
:1010500010936000112309F0A8959FBF1F91089578
:10106000382F20E08091350590913605822793270F
:1010700040E061E270E19C01220F331F97FF04C042
:10108000C9018627972701C0C9014F5F483099F7EA
:101090009093360580933505089587E38093D003B8
:1010A00080E092ECA1E0B0E08093D1039093D20372
:1010B000A093D303B093D40387E08093DD0380EC47
:1010C00092E9ADEEB9E18093D5039093D603A09356
:1010D000D703B093D80385E08093DE038DEE9EEFB7
:1010E000ADEABEED8093D9039093DA03A093DB03BE
:1010F000B093DC03AFEDB3E080E090E0863010F019
:10110000E0E004C0FC01EF57FC4FE081ED93019655
:101110008831910599F782E08093F7038AE0809304
:10112000F803089580EC91EDA8E9BBE180939D035D
:1011300090939E03A0939F03B093A00380E090E060
:10114000A0E0B0E58093A1039093A203A093A30332
:10115000B093A403E5EAF3E080E081938F5F8031F0
:10116000E1F708958436910520F4BC0180E090E019
:1011700025C08E3B910550F48A559040BC0180E01B
:1011800090E02AE030E040E050E016C0823D91055A
:1011900050F4845B9040BC0180E090E024E630E0B5
:1011A00040E050E009C08D5C9040BC0180E090E0E0
:1011B00028E532E040E050E00E947A2F24E630E05B
:1011C00040E050E00E947A2F089590E08C599F4FA4
:1011D0000E94B2080895DC019896EC91F0E0E77067
:1011E000F070E758FC4F808108958F929F92AF92E4
:1011F000BF92CF92DF92EF92FF920F931F938C01D9
:101200000E94EB08D80197962C9130E043E150E022
:10121000249FF001259FF00D349FF00D1124EB5415
:10122000FD4F80809180A280B38090E00F96AA2726
:1012300097FDA095BA2FBC01CD0120E43FE14DE719
:1012400050E00E947A2FA50194010E94AC2F690101
:101250007A0180ED97E0A0E0B0E0C80ED91EEA1E4A
:10126000FB1ED80198968C91887181F060E07EEE2B
:101270008AEB9BE0A50194010E94AC2F28513C4FC2
:101280004F4F5F4FC20ED31EE41EF51E87EE93E054
:10129000A0E0B0E0C80ED91EEA1EFB1EC701B601D1
:1012A00028EE33E040E050E00E94AC2FCA01B901C3
:1012B00028EE33E040E050E00E947A2F1F910F911A
:1012C000FF90EF90DF90CF90BF90AF909F908F9066
:1012D00008958F3F910509F010F480E0089522E011
:1012E0008030920710F481E008958050934010F010
:1012F00083E0089582E00895CF92DF92FF920F93EA
:101300001F93CF93DF93F82FEB016A01182F1695E7
:10131000E0E088819981D6018C938A819B81119626
:101320008C9311978C819D8112968C9312978E814C
:101330009F8113968C931397288139814A815B8111
:101340006C817D818E819F819295990F990F907C00
:10135000832F8370982B852F8370880F880F982B8D
:10136000872F83708295807F982B14969C9385E0BD
:1013700090E0C80ED91E2896EF5F1E1750F6F0FFBA
:1013800021C0888199810E946909F82E8A819B81F8
:101390000E946909182F8C819D810E946909082F7C
:1013A0008E819F810E946909F294FF0CFF0C70EC02
:1013B000F7221295107F1F29182B000F000F012B09
:1013C000D6010C93DF91CF911F910F91FF90DF9089
:1013D000CF90089523E08032920718F420E030E0A7
:1013E00026C023E0883E920748F49C012F513340E9
:1013F00054E0369527955A95E1F719C027E0803DCE
:10140000920720F49C012C5D334011C028E08839FC
:10141000920718F02FEF33E00AC09C01285C374098
:1014200044E0369527954A95E1F72D503C4FC90188
:1014300008958C30910548F49C0174E0220F331F0D
:101440007A95E1F7285D3C4F17C023E0843F92076F
:1014500020F49C0124523C4F0FC024E080309207BE
:1014600018F020E938E008C09C012657334F64E0AB
:10147000220F331F6A95E1F7C90108959C01369543
:10148000279525753575821B930B9C0136952795FD
:10149000369527952373337383739373280F391FFE
:1014A000C901E4E096958795EA95E1F7820F931FCD
:1014B0008F709F7021E031E0AC01429FC001439FDB
:1014C000900D529F900D1124892F0895882339F093
:1014D0002D9800002B9A00002D9A000008952D9859
:1014E00000002B9800002D9A000008952D9A00000E
:1014F00083B12D98000090E0B4E096958795BA9559
:10150000E1F7817008950F931F93082F5C9A2D982F
:101510005C9810E0802F80780E94660A000F1F5FA1
:101520001830C1F72D981F910F9108958F770E9461
:10153000830A08950F931F93082F10E0802F80785F
:101540000E94660A000F1F5F1830C1F72D981F9187
:101550000F9108950F931F932D9880E000E0182FAE
:10156000110F0E94760A810F0F5F0830C1F71F919B
:101570000F9108950E94960A0E94AA0A5C9A089503
:101580001F93162F80680E94830A812F0E949A0A57
:101590005C9A1F9108951F931091D9031827E0EDCD
:1015A000F3E0E80FF11D89E767850E94C00A8DE32B
:1015B000612F0E94C00A82E4612F0E94C00A1F911D
:1015C000089586E20E94BA0A08950F931F938C0132
:1015D0008CE1F80164810E94C00A8DE1F801658107
:1015E0000E94C00A8EE1F80166810E94C00A80E272
:1015F000F80167810E94C00A81E2F80160850E94BB
:10160000C00A82E2F80161850E94C00A83E2F80103
:1016100062850E94C00A84E2F80163850E94C00AC4
:1016200085E2F80164850E94C00A8AE2F8016585B6
:101630000E94C00A8EE6F80166850E94C00A8FE605
:10164000F80167850E94C00A80E7F80160890E945E
:10165000C00A81E7F80161890E94C00A82E7F801A7
:1016600062890E94C00A1F910F910895EF92FF9224
:101670000F931F93CF93DF937B018C01603028E39E
:1016800072072CE982072CE1920728F520E836E959
:1016900048E950E00E94AC2FE9016897B90180E069
:1016A00090E020E839E647E65FEF0E947A2F6E0D62
:1016B0007F1D801F911F32E0660F771F881F991FC3
:1016C0003A95D1F721E732E040E050E00E94AC2F9C
:1016D000890180E421C020E03DE241E351E00E9425
:1016E000AC2FE9016897B90180E090E020E033ED8C
:1016F0004EEC5EEF0E947A2F6E0D7F1D801F911FB2
:10170000660F771F881F991F21E732E040E050E005
:101710000E94AC2F890180E69E012F71622F680F15
:1017200085E70E94C00A86E7612F0E94C00A87E70A
:10173000602F0E94C00ACDB7DEB7E6E00C941130EE
:10174000682F8DE60E94C00A08959F92AF92BF92C3
:10175000CF92DF920F93DF93CF9300D000D0CDB71D
:10176000DEB7982E83E00E94BA0A8093F90384E0E2
:101770000E94BA0A8093FA0386E060E00E94C00AE1
:1017800087E061E00E94C00A89E06FE70E94C00A1A
:101790008AE065E00E94C00A8BE062E10E94C00A14
:1017A0008CE065E10E94C00A8DE06DEF0E94C00AE6
:1017B0008EE060E00E94C00A992019F084E193E075
:1017C00008C08091F70323E1829FC00111248B544C
:1017D0009D4F0E94E50A80E36CE80E94C00A82E304
:1017E0006FE00E94C00A83E362E40E94C00A84E3BF
:1017F0006AE00E94C00A85E36AE20E94C00A86E3AA
:101800006DE20E94C00A87E364ED0E94C00A88E38B
:1018100060E00E94C00A89E360E00E94C00A99204B
:1018200049F065E8A62E61ECB62E61ECC62E6EED91
:10183000D62E08C0A090D903B090DA03C090DB0385
:10184000D090DC030AE38D2D9927AA27BB27898333
:101850009A83AB83BC83802F69810E94C00A802F4A
:101860008B5F69810E94C00ADC2CCB2CBA2CAA2485
:101870000F5F0E3341F783E46FEF0E94C00A84E4E8
:101880006FEF0E94C00A85E46FEF0E94C00A86E4F1
:101890006FEF0E94C00A992019F08DE666E003C040
:1018A0008DE66091DD030E94C00A89E760E00E9436
:1018B000C00A8AE76091DE030E94C00A83E760E005
:1018C0000E94C00A84E760E00E94C00A992029F0C3
:1018D00060EC72E98DEE99E108C06091D5037091DA
:1018E000D6038091D7039091D8030E94360B0F90B6
:1018F0000F900F900F90CF91DF910F91DF90CF90CD
:10190000BF90AF909F90089587E061E00E94C00A69
:101910008EE764E20E94C00A88E063E00E94C00A89
:1019200088E060E00E94C00A87E065E00E94C00A8B
:1019300085E062E00E94C00A83E00E94BA0A8093B8
:10194000F90384E00E94BA0A8093FA030895582F9D
:1019500040919E04842F90E0FC01EF70F0709F0195
:101960002F5F3F4F74E0959587957A95E1F728179B
:10197000390751F0E257FB4F5083842F8F5F8F70F0
:10198000407F842B80939E0408951F920F920FB680
:101990000F9211241F932F933F934F935F936F9355
:1019A0007F938F939F93AF93BF93CF93DF93EF93E7
:1019B000FF93C0918600D09187002091E20430917E
:1019C000E3048091C104882309F062C0BE01621B58
:1019D000730B2091A1033091A2034091A303509176
:1019E000A40325FD02C07695679589E0653C7807DC
:1019F000B8F1809147031CE1569547953795279597
:101A00001A95D1F7211531054105510521F421E041
:101A100030E040E050E090E0A0E0B0E02817390767
:101A20004A075B07D0F4809147038F3FB1F020E075
:101A30000EC0E22FF0E0EE0FFF1FDF01AE53BB4FF1
:101A40008D919C91E95DFC4F918380832F5F809104
:101A50004703281770F31092C0041092470318C070
:101A600082E06D3B780760F180914703803140F55B
:101A700010914703CB010E94EA09E12FF0E0EE0F3D
:101A8000FF1FEE53FB4F918380831F5F109347032B
:101A9000D093E304C093E204FF91EF91DF91CF91E3
:101AA000BF91AF919F918F917F916F915F914F9176
:101AB0003F912F911F910F900FBE0F901F9018957F
:101AC0008FEF80934703E4CF83E0809380008AE91F
:101AD000809381008091A10386FD05C080918100E3
:101AE0008064809381008FEF9FEF909389008093B3
:101AF000880080916F00806280936F0008956F303E
:101B000018F086958058089589E0689F802D1124EB
:101B10000895882319F460E071E002C063E071E089
:101B200089E396E00E942E2D0895A0E0B0E0EBE955
:101B3000FDE00C94F32F182F0E94DF299B01AC01CC
:101B400080912F0590913005A0913105B09132051B
:101B500069017A01C81AD90AEA0AFB0AD701C60143
:101B600089589341A040B04010F010922E05209368
:101B70002F05309330054093310550933205209165
:101B8000C104822F81508230E8F580912E05882390
:101B900009F44FC1813011F482E0BCC1803108F0FA
:101BA00035C1E82FF0E0EE53FB4F10838F5F809339
:101BB0002E05803109F0B0C1A4ECB4E0213039F435
:101BC0001196EC911197E695E6958C9109C08D914F
:101BD0009C911197E92FE695E695E6959695879560
:101BE000E03140F4F0E090E0EE0FFF1FE95DFC4FC4
:101BF000918380831092C004129684E0A23DB807BE
:101C0000E9F68AC1233009F004C180912E058823AA
:101C100021F41F3009F080C10CC1883130F4E82F65
:101C2000F0E0EF53FB4F108374C1883109F0EEC030
:101C3000112309F0EBC0C0E0D0E00BE010E0DE01C2
:101C400063E0AA0FBB1F6A95E1F7C09FB001C19F77
:101C5000700DD09F700D1124FB01EE53FB4F80815E
:101C60002181922F977095958795FD01EE0FFF1FAB
:101C7000E95DFC4F91838083FB01ED53FB4F308185
:101C80003695369536952181422F4295440F407EF8
:101C9000842F832B269526952695922F97709595C0
:101CA0008795FD01EE0FFF1FE75DFC4F9183808359
:101CB000FB01EC53FB4F808182958695869583705E
:101CC0004181942F990F990F292F282B42954695E2
:101CD0004695437082818170880F880F382F342B8E
:101CE00035952795FD01EE0FFF1FE55DFC4F318314
:101CF0002083FB01EA53FB4F308136952181422F2F
:101D0000479544274795842F832B2695922F9770CC
:101D100095958795FD01EE0FFF1FE35DFC4F9183C5
:101D20008083FB01E953FB4F308132953F70218165
:101D3000422F4295407F842F832B22952F70922F24
:101D4000977095958795FD01EE0FFF1FE15DFC4FA4
:101D500091838083FB01E853FB4F8081881F882794
:101D6000881F4181942F990F292F282B441F442726
:101D7000441F82818370880F382F342B3595279527
:101D8000FD01EE0FFF1FEF5CFC4F31832083FB0151
:101D9000E653FB4F3081369536952181422F42958F
:101DA000440F440F407C842F832B26952695922F39
:101DB000977095958795AA0FBB1FFD01ED5CFC4FB1
:101DC0009183808365537B4FFB012081229526956B
:101DD00027704181342F330F330F330F832F822B22
:101DE000942F92959695977095958795AB5CBC4F7F
:101DF00011969C938E932196C230D10509F01FCF86
:101E00008091D80483FD02C01092C00410922E0568
:101E100083C0243009F080C040912E05442359F43A
:101E2000183AB1F4109236051092350588EA0E94EE
:101E3000300881E06FC0413019F41093330504C0BD
:101E4000423031F410933405812F0E9430085DC078
:101E500060913405262F30E0220F331FE42FF0E08D
:101E6000C90102968E179F0734F0433268F7E15498
:101E7000FB4F1083E9CF2D5F3F4F409135055091C7
:101E80003605E217F30749F4912F80E048275927D8
:101E9000509336054093350538C0812F90E04817A0
:101EA000590789F580913305813069F5613118F062
:101EB00080E180933405D090340542ECE42E44E078
:101EC000F42E00E010E01BC0F701D081C0E081815A
:101ED00090E08C2B9D2B33E0969587953A95E1F712
:101EE0000E94EA09F801EE0FFF1FE95DFC4F9183A4
:101EF00080830F5F1F4F82E090E0E80EF91E0D1502
:101F000018F31092C00410922E0580912E0588239C
:101F100019F08F5F80932E05CDB7DEB7E8E00C9403
:101F20000F30FF920F931F93CF93DF93182F092F3A
:101F3000F62E8EE30E94C00A212F302FC901EC013A
:101F400010E005C08FE769910E94C00A1F5F1F154E
:101F5000C8F385E064E00E94C00A83E00E94BA0AE8
:101F60008093F90384E00E94BA0A8093FA030E94E6
:101F7000DF296093FB037093FC038093FD03909330
:101F8000FE0387E069E00E94C00A81E080939A0323
:101F9000CDB7DEB7E5E00C9412300E94910F80912E
:101FA0009A038130D9F40E94DF292091FB033091FC
:101FB000FC034091FD035091FE03621B730B840BE5
:101FC000950B605A76488140904040F4E8CF89E311
:101FD00096E067E071E00E942E2D089580919A03AB
:101FE0008130A9F3089589E396E06EE70E94E62E1A
:101FF0000895A0E0B0E0EFEFFFE00C94F22F6C0149
:1020000089E396E06EE70E94E62E760100E010E09C
:10201000C0E0D0E0B0E2BB2E0AC00830110521F4C8
:102020009E012095F60120870894E11CF11CF70120
:102030006081862F8D57823040F489E396E06DE70A
:102040000E94E62EF70160816B2589E396E00E94ED
:10205000E62E0115110551F0F70180819E01280F30
:10206000311DC32FDD27C20FD31FD0700F5F1F4F4D
:102070000930110591F6CDB7DEB7E9E00C940E30CA
:10208000A9E0B0E0E6E4F0E10C94F92F382FE62F58
:102090008091A30490E0019664E270E00E94992F81
:1020A000982F8093A30488E9898380E18A83913003
:1020B00071F0913028F0923099F09330E1F416C02D
:1020C00085E08B8381EF8C832F5F2D8317C09B83EB
:1020D00081EF8C8384E6489FC00111249D830EC04C
:1020E00084E08B8381EF8C833D8308C09B8381EFE9
:1020F0008C83ED8303C00E94F30F04C0CE010196D0
:102100000E94F90F2996E2E00C9415300F931F936B
:10211000CF93DF93182F092F89E396E06EE70E9493
:10212000E62E212F302FC901EC0110E000E288815A
:102130008D57823040F489E396E06DE70E94E62EE9
:1021400088818027888389E396E069910E94E62E42
:102150001F5F193061F789E396E06EE70E94E62E73
:10216000DF91CF911F910F910895A9E0B0E0EBEBC3
:10217000F0E10C94F92F382F8091A304882379F48F
:102180008EEF89833A836B83842F90E095958795B2
:102190008C832D83198618861F821E822FC0409142
:1021A0009E04842F90E09C012F70307054E0959530
:1021B00087955A95E1F78217930721F18DEF89836F
:1021C0001A821B82DE01149620E008C0E257FB4F02
:1021D00080818D93405F2F5F263069F0842F90E0DF
:1021E000FC0134E0F595E7953A95E1F78F70907032
:1021F000E817F90759F740939E042A83CE01019608
:102200000E9486108091A30490E0019666E070E041
:102210000E94992F8093A3042996E2E00C94153034
:102220009F92AF92BF92CF92DF92EF92FF920F9365
:102230001F93B82EA62ED42EC22E902E0E94DF29D8
:102240007B018C0180918D0420919F043091A0042A
:102250004091A1045091A2048823B1F0D801C70194
:10226000821B930BA40BB50B815E9E42A040B04035
:1022700020F12C2DDC1408F42D2D8B2D6A2D422FEE
:10228000292D0E94401011C0D801C701821B930B59
:10229000A40BB50B81539547A040B04070F08B2D37
:1022A0006A2D4D2D2C2D0E94B510E0929F04F092C6
:1022B000A0040093A1041093A2041F910F91FF901A
:1022C000EF90DF90CF90BF90AF909F90089589E3FB
:1022D00096E0609100040E94E62E08951F93182F47
:1022E00089E396E0612F0E94E62E80910004812709
:1022F000809300041F9108951F93192F0E946E115F
:10230000812F0E946E111F910895DF92EF92FF922C
:102310000F931F93D82E7B011092000409E316E05F
:10232000C80165EB0E94E62EC80162E60E94E62E17
:102330008D2D0E946E11C7010E947C111F910F917B
:10234000FF90EF90DF900895E82FF0E0E456FC4F07
:10235000E185E03158F4F894F0E0EE0FFF1FE95DFD
:10236000FC4F0190F081E02D78940DC0E03129F010
:10237000E13129F0E0E0F2E006C082E101C083E152
:102380000E94332BFC01CF0108958CE060E00E9495
:10239000642A8BE061E00E94642A8DE061E00E9483
:1023A000642A82E060E00E94642A84E061E00E9486
:1023B000642A0895892B19F08FE061E002C08FE054
:1023C00060E00E94D02A0895A0E2B0E0EAEEF1E1D8
:1023D0000C94F12F8CE00E94BA0A882389F589E3D6
:1023E00096E063E171E00E942E2D5E9A409A80E0B3
:1023F0000E94A50B0E94840C5E98409821C089E33E
:1024000096E00E94AD2E482F8091C104882321F0D0
:10241000842F0E94950D14C080912C05E82FF0E0C8
:1024200031969F012F713070319780912B0590E08C
:102430002817390729F0EE5FFA4F408320932C05C7
:1024400089E396E00E94732E892BC9F680919A0346
:10245000843009F08EC00E94DF296093B00470932D
:10246000B1048093B2049093B304611571058105A2
:10247000910561F481E090E0A0E0B0E08093B004C9
:102480009093B104A093B204B093B3048091BC04C0
:102490009091BD0481609093BD048093BC0483E05F
:1024A00080939A038FE70E94960A09EF14E00E9436
:1024B000AA0AF80181938F01F5E002301F07B9F7EE
:1024C0004091E4048091F904282F30E0842F90E0BB
:1024D0008227932786FF40C080E448274093E40486
:1024E000C90188739070C89709F510E014C01F5F88
:1024F0008091F803E12FF0E084FF06C0E750FB4F26
:1025000080810E94A70C07C0E750FB4F89E396E04B
:1025100060810E94E62E212F30E08091F90490E046
:10252000877090708217930714F716C02F7330705E
:10253000232B91F48091FA048093B4048091FB04DE
:102540008093B6048091FC048093B7048091FF04CB
:102550008093BE041092BF0480912D05813019F440
:1025600082E080932D0580912D05833011F4109227
:102570002D050E94DF295B016C018091B8049091C8
:10258000B904A091BA04B091BB040097A105B105AC
:10259000C9F086017501E81AF90A0A0B1B0BD8016C
:1025A000C701885B9B40A040B04060F00E94E10AF8
:1025B0008093B5041092B8041092B9041092BA0432
:1025C0001092BB0480ED93E00E94F5082091AC04CA
:1025D0003091AD044091AE045091AF048601750175
:1025E000E21AF30A040B150BE616F706080719079B
:1025F00008F428C1A092AC04B092AD04C092AE041D
:10260000D092AF04A8958091C0048830A0F080914A
:10261000A1039091A203A091A303B091A403FCE1B4
:10262000B695A79597958795FA95D1F70097A10547
:10263000B10509F0A7C18091C0048F5F8093C004E9
:10264000E090B004F090B1040091B2041091B30492
:10265000E114F1040105110511F180ED93E00E94F0
:10266000F508AE18BF08C00AD10A6A157B058C05AB
:102670009D0588F48091A10384FD04C080ED97E05E
:102680000E94DA111092B0041092B1041092B204B8
:102690001092B30404C080E090E00E94DA1190919F
:1026A000E404907C9093E40400912C0510912B0598
:1026B0000117B1F180912D05823091F590589093DA
:1026C000E40480ED93E00E94EB08893010F048E0CC
:1026D00002C0482F415030E013C03F5FA32FB0E04D
:1026E000812F90E0FC01EE5FFA4F2081FD01EC515B
:1026F000FB4F2083AE5DBA4F2C930196182F1F71AC
:10270000341710F4101749F710932B05832F895CA9
:102710009091E404892B8093E404309322051AC03D
:1027200020912D052430D1F490912205E3E2F5E0CB
:10273000A5EEB4E0292F30E02E0F3F1F02C081919B
:102740008D93E217F307D9F7995C8091E404982BF5
:102750009093E40483E080932D0538C08091A70412
:10276000823061F491609093E4045E9A409A05EAA5
:1027700013E07E010894E11CF11C11C09093E40465
:102780005E984098222319F481E080932D05809172
:102790002D05833061F784E080932D05E8CFF801A3
:1027A00081918F010E94A411F701819391937F0180
:1027B000F3E0053B1F0799F78091F8038770BE018E
:1027C0006F5F7F4F45EE54E00E947C095D9A419A0D
:1027D0002091A5042223A1F09091DD03992381F09B
:1027E0008091A6048F5F8093A6048150821729F4FC
:1027F0001092A604892F815001C0892F0E94A00B3E
:102800008091A4040E94CB0A80ED93E00E94EB0823
:10281000682F84EE94E00E94910FE091A404EF5F92
:10282000E093A404E83131F0F0E0E053FC4F8785F9
:10283000882341F41092A40405C05E9A409A89E06E
:102840008093C0048091F803887171F180919A039C
:10285000823051F58091BC049091BD04880F991F7E
:102860009093BD048093BC0483E080939A030E94FC
:10287000840C0E94DF296093B8047093B90480939C
:10288000BA049093BB04611571058105910561F44B
:1028900081E090E0A0E0B0E08093B8049093B904A8
:1028A000A093BA04B093BB048091F80384FF1EC0C8
:1028B0008091BC049091BD048E7F0E943E0A182F27
:1028C0008091B4046091BE040E947F0D082F809116
:1028D000B504612F0E947F0D282F8091B60460916E
:1028E000B704402F00919B030E9410115D984198FE
:1028F0008091A7048130D1F0813020F0823009F03E
:1029000047C034C083E10E94032B892B09F040C0EB
:1029100081E08093A7040E94D1296093A80470935A
:10292000A9048093AA049093AB0432C083E10E946F
:10293000032B892B21F50E94D1292091A8043091E5
:10294000A9044091AA045091AB04621B730B840B41
:10295000950B695E734080409040D0F082E0809398
:10296000A70480ED97E00E94DA1112C083E10E9473
:10297000032B892B69F080E090E00E94DA1110921D
:10298000A70406C08091C004883009F058CF55CF05
:10299000A096EAE00C940D308FE061E00E94642A7A
:1029A0008FE060E00E94D02A08951F93182F0E94A4
:1029B000DF2960939F047093A0048093A1049093F7
:1029C000A20410938D04112329F440E855E260E03D
:1029D00070E004C040E051EE60E070E089E396E012
:1029E0000E94EC2D1F910895ACE1B0E0EAEFF4E114
:1029F0000C94F12F0E94DF297B018C0181E00E9461
:102A0000A50B84E7A82E6E010894C11CD11CB3E06D
:102A1000BB2EA982C60161E00E94CD0FB0929A033D
:102A20000E94840C6AEF70E080E090E00E94052A2A
:102A300080919A03833009F07DC089E396E00E947B
:102A4000732E892B09F076C00E94DF296E197F0949
:102A5000800B910B6058734C894C914008F06AC010
:102A6000D8CF8FE70E94960A0E94AA0A843509F0FF
:102A70005CC089830E94AA0A182F00E010932404E6
:102A8000009323040E94AA0A080F111D1093240426
:102A9000009323040E94AA0A809322040E94AA0A97
:102AA00080932104813108F040C0FF2407C00E94B8
:102AB000AA0A0F5F1B4FF8018083F3940F2D10E0DB
:102AC0008091210490E0880F991F0817190778F367
:102AD00080E78983CE01019661E00E94CD0F83E0FB
:102AE00080939A030E94840C62E370E080E090E09F
:102AF0000E94052A80919A038330A9F08FE70E94F3
:102B0000960A0E94AA0A803581F4898305EB13E0B6
:102B10000E94AA0AF80181938F01F3E0003D1F078C
:102B2000B9F781E003C082E001C083E06C96EAE07F
:102B30000C940D3080919A03833009F092CFF3CF3B
:102B400083E00E94BA0A8093F90384E00E94BA0AE3
:102B50008093FA0387E061E00E94C00A6AE070E0B7
:102B600080E090E00E94052A0E94840C00000895F5
:102B70000F931F93082F19C05E9A409A64E670E085
:102B800080E090E00E94052A5E98409864E670E03C
:102B900080E090E00E94052A1F5F101768F36CE246
:102BA00071E080E090E00E94052A10E0F6CF482F07
:102BB000392F25E00DC0F999FECF1FBA842F932F2E
:102BC00092BD81BD60BD0FB6F894FA9AF99A0FBE16
:102BD000215059F0F999FECF842F932F92BD81BDDA
:102BE000F89A80B5681739F7089582E00E94B81501
:102BF0000895A0E0B0E0EFEFF5E10C94EA2F482E45
:102C0000562EEE24FF2488249924C0E0D0E0CC2462
:102C1000DD2476E4372E04C0CC24DD2455245394DF
:102C2000442069F480919B03839DE00111246CE9A9
:102C3000E62E63E0F62E59E1852E912C1DC021E091
:102C4000421671F480919B03839DE00111246B96E1
:102C500040EDE42E43E0F42E39E2832E912C0CC09B
:102C600032E0431649F42BE9E22E23E0F22E91E004
:102C7000892E912CC8E1D1E03E016C0C7D1C109294
:102C8000360510923505E3011BC0552059F4F9991A
:102C9000FECFD2BDC1BDF89A80B5F701E00FF11F9C
:102CA000808307C0F701E00FF11FCE0160810E9411
:102CB000D7150E0D1F1DF80180810E943008219646
:102CC0009E012619022F10E008151905F0F2CE0119
:102CD0005520D9F4F999FECFD2BDC1BDF89A20B5DF
:102CE000F999FECF2196D2BDC1BD2197F89A80B542
:102CF00090E0B22EAA248A299B2920913505309193
:102D000036052817390759F487CF21966091360583
:102D10000E94D715CE01609135050E94D71580E23B
:102D200091E0C80ED91E91EEC91692E0D90608F4BA
:102D300077CF852DCDB7DEB7E1E10C94063080E08A
:102D400061E00E94F91581E061E00E94F9150895A3
:102D500082E061E00E94F915089582E060E00E943F
:102D6000F91580919B03843020F010929B030E9400
:102D7000A81608951F93182F0E94AD1680919B03EB
:102D8000811731F0143020F410939B030E94A81691
:102D90001F91089510928B0485E6E6E2F4E0DF01CE
:102DA0001D928A95E9F708951F93182F8F3711F018
:102DB0008830E1F5E0918B04EE2309F455C0E15031
:102DC000E0938B04F0E0EA5DFB4F108289E396E02C
:102DD0006DE00E94E62E10E00AC0E12FF0E0EA5D0F
:102DE000FB4F89E396E060810E94E62E1F5F809191
:102DF0008B04181790F389E396E060E20E94E62EB8
:102E000089E396E06DE00E94E62E10E00AC0E12F13
:102E1000F0E0EA5DFB4F89E396E060810E94E62ED8
:102E20001F5F80918B04181790F31CC08B3119F42D
:102E30000E94CA161FC08D30E9F08A30D9F0809107
:102E40008B04843688F489E396E0612F0E94E62E95
:102E500080918B04E82FF0E0EA5DFB4F10838F5FD9
:102E600080938B0480E007C089E396E067E00E94CE
:102E70009A2BF8CF81E01F9108951F93CF93DF9392
:102E8000CFEDD3E010E03BC089E396E062E271E071
:102E90000E942B2D89E396E0612F4AE050E00E94CA
:102EA000A82C89E396E06FE271E00E942B2D6991D6
:102EB00070E080E090E02091DE0330E040E050E000
:102EC0000E947A2F20E137E240E050E00E947A2F02
:102ED000DC01CB014091D5035091D6036091D7031B
:102EE0007091D803480F591F6A1F7B1F89E396E032
:102EF0002AE030E00E946F2C1F5F183119F08881A2
:102F0000882311F6DF91CF911F910895EF92FF92E0
:102F10000F931F93882339F489E396E061E77AE001
:102F20000E94B82B3BC090E00E94B20824E630E03B
:102F300040E050E00E94AC2F122F032FF42EE52E1C
:102F4000622F732F842F952F2AE030E040E050E06D
:102F50000E94AC2F89E396E0BA01A9012AE030E093
:102F60000E94602C89E396E06EE20E949A2B612F0A
:102F7000702F8F2D9E2D2AE030E040E050E00E941F
:102F8000AC2FAB01BC0189E396E02AE030E00E945F
:102F9000602C89E396E063E70E94CC2B1F910F9190
:102FA000FF90EF900895FF920F931F93CF93DF93BD
:102FB00089E396E067E67AE00E94792B8091B50379
:102FC000813041F489E396E06EE47AE00E94B82B08
:102FD000FF246DC0823029F489E396E067E37AE04C
:102FE000F5CF843029F489E396E063E27AE0EECF0E
:102FF000853071F789E396E068E17AE0E7CFCF2D7D
:10300000D0E0C930D1051CF06F2D685C02C06F2D77
:103010006F5C89E396E00E949A2B89E396E060E179
:103020007AE00E94792BBE016F5F7F4F89E396E0C3
:103030004AE050E00E94042D89E396E065E07AE0E2
:103040000E94792B8E010B541C4FD8011196EC91E4
:10305000E032F8F489E396E068EF79E00E94792B9A
:10306000F8018181803130F089E396E063E371E01B
:103070000E942B2DCB54DC4F698170E06F70707013
:103080006F5F7F4F89E396E04AE050E00E94172D82
:103090000DC0F0E0EF70F070EE0FFF1FE75BFC4F2C
:1030A0006081718189E396E00E942E2DF3948091D6
:1030B0002204F81608F4A3CF89E396E06DED79E0D9
:1030C0000E94792B8091CD030E94861789E396E0B8
:1030D00062EC79E00E94792B8091CE030E948617E2
:1030E00089E396E067EA79E00E94792B8091CF032B
:1030F0000E94861789E396E06CE879E00E94792BBC
:103100004091C5035091C6036091C7037091C803F5
:10311000411551056105710539F189E396E02AE011
:1031200030E00E946F2C89E396E069E579E00E9427
:10313000792B8091C9030E94E508AB01BC0189E3AA
:1031400096E02AE030E00E946F2C89E396E065E388
:1031500079E00E94792B89E396E06091CA034AE006
:1031600050E00E94BA2C06C089E396E06CE279E058
:103170000E94B82B89E396E06FE079E00E94792BFA
:103180006091CB037091CC0389E396E04AE050E074
:103190000E94942C89E396E062EF78E00E94792BFC
:1031A0006091C403603450F470E06F5F7F4F89E337
:1031B00096E04AE050E00E94172D06C089E396E0B1
:1031C00069EE78E00E94B82B89E396E06CEC78E039
:1031D0000E94792B8091C30380FD03C065E371E0F9
:1031E00002C069E371E089E396E00E942E2D89E335
:1031F00096E06FEA78E00E94792B8091C303827099
:103200000E94890D89E396E060E978E00E94792BBD
:103210008091C30384700E94890D89E396E061E781
:1032200078E00E94792B8091C30388700E94890DF9
:10323000CDB7DEB7E5E00C9412301F93CF93DF9348
:1032400089E396E06BEB7BE00E94792B4091D503FC
:103250005091D6036091D7037091D80389E396E02B
:103260002AE030E00E946F2C89E396E065EA7BE07B
:103270000E94792B4091D9035091DA036091DB03CE
:103280007091DC0389E396E020E130E00E946F2C2E
:1032900089E396E06FE87BE00E94792B89E396E072
:1032A0006091DD034AE050E00E94BA2C89E396E089
:1032B00069E77BE00E94792B89E396E06091DE0369
:1032C0004AE050E00E94BA2C89E396E063E67BE096
:1032D0000E94792BCFEDD3E010E012C0112331F022
:1032E00089E396E06DE371E00E942B2D89E396E07F
:1032F00069914AE050E00E94A82C1F5F183119F034
:103300008881882359F789E396E00E94A22B89E3FC
:1033100096E06DE47BE00E94792B89E396E0609172
:10332000F7034AE050E00E94BA2C89E396E068E394
:103330007BE00E94792BE091F803F0E0E770F070F9
:10334000EE0FFF1FE759FC4F6081718189E396E022
:103350000E942E2D89E396E063E27BE00E94792BA8
:103360008091F80390E0887190708830910589F021
:10337000893091051CF4892B39F01BC080319105EF
:1033800069F04897B1F40FC089E396E06AE17BE009
:103390000EC089E396E06EE07BE009C089E396E029
:1033A00068E07BE004C089E396E06EEF7AE00E947B
:1033B000B82B89E396E06AEE7AE00E94792B40917F
:1033C000D1035091D2036091D3037091D40389E368
:1033D00096E02AE030E00E946F2C89E396E061EDF0
:1033E0007AE00E94792B8091A10380710E94890D5F
:1033F00089E396E068EB7AE00E94792B8091A10343
:1034000080740E94890D89E396E06FE97AE00E945A
:10341000792B8091A10380720E94890D89E396E047
:1034200062E87AE00E94792B80ED93E00E94F50833
:10343000AB01BC0189E396E02AE030E00E94602CF9
:1034400089E396E06DE77AE00E94792B80ED93E0C6
:103450000E94F5089B01AC0160E472E48FE090E00B
:103460000E94AC2F89E396E0BA01A9012AE030E07E
:103470000E94602C89E396E06AE77AE00E94B82B0C
:10348000DF91CF911F910895EF92FF920F931F93B9
:103490007C0109E316E0C8016F2D70E04AE050E0BE
:1034A0000E94832CC8016EE20E949A2BB70184E02F
:1034B000769567958A95E1F76F707070C8014AE05C
:1034C00050E00E94832CC8016EE20E949A2B8FE08C
:1034D000E822FF24C801B7014AE050E00E94832C93
:1034E0001F910F91FF90EF9008950F931F93CF932B
:1034F000DF93209125042F3FA9F589E396E061EF42
:1035000075E00E94792B83E793E00E94441A89E3D7
:1035100096E060ED75E00E94792B809123049091F4
:1035200024040E94441A89E396E06DE975E00E9444
:10353000B82B89E396E06AE775E00E94B82B89E32F
:1035400096E062E675E00E94B82B89E396E06DE3B1
:1035500075E00E94B82B89E396E00E94A22B0E949E
:10356000D31769C012160CF066C0332727FD3095BB
:103570008091220490E0821793070CF45CC089E3E9
:1035800096E068E275E00E94792B60912504772728
:1035900067FD709589E396E04AE050E00E94172DA0
:1035A00089E396E06DEF74E00E94792B08E210E069
:1035B0003AC0C12FD0E0CC0FDD1FCF5FDB4F288199
:1035C00030E080912504992787FD90950197281771
:1035D000390741F589E396E06FE371E00E942B2DF6
:1035E00089E396E0602F4AE050E00E94A82C89E32E
:1035F00096E063E471E00E942B2DE981F0E0EF702A
:10360000F070EE0FFF1FE75BFC4F6081718189E373
:1036100096E00E942B2D89E396E067E471E00E941A
:103620002B2D0F5F1F5F80912104181710F289E383
:1036300096E00E94A22BDF91CF911F910F910895E8
:10364000ACE1B0E0E6E2FBE10C94F32F282F80918F
:1036500025048F3F09F03BC1822F90E0FC013A978F
:10366000EF36F10508F02CC1EC5CFF4F0C942030D4
:1036700089E396E069E471E0A7C089E396E065E537
:1036800071E00E942E2D85E78983DE011296E5EB1D
:10369000F3E08BE101900D928150E1F7CE010196AC
:1036A0006CE10E94CD0F0E94840C83E080939A030A
:1036B00068EC70E080E090E00E94052A80919A0317
:1036C000843009F0FDC08FE70E94960A0E94AA0A82
:1036D0008983853509F0F4C089E396E06FED74E0E5
:1036E0000E94B82B89E396E061EC74E00E94B82B4D
:1036F00089E396E063EA74E0ACC089E396E06DE6A6
:1037000071E00E942E2D89E68983CE01019661E049
:103710000E94CD0F0E94840C83E080939A0368EC92
:1037200070E080E090E00E94052A80919A03843046
:1037300009F0C6C08FE70E94960A0E94AA0A8983F0
:103740008E010E5F1F4FBDE1EB2EF12CEC0EFD1E26
:103750000E94AA0AD8018D938D01AE15BF05C1F74D
:10376000A5EBB3E0FE0132968BE101900D92815002
:10377000E1F78981893409F0A3C089E396E065E81F
:1037800074E00E94B82B89E396E067E674E00E943B
:10379000B82B89E396E069E474E05BC089E396E0C6
:1037A00067E871E00E942E2D8EEF8093250488C07B
:1037B00020522750922F905380912204891738F479
:1037C00089E396E066E971E00E942E2D79C090931E
:1037D00025046FC084E18093250489E396E062E1CB
:1037E00074E037C085E18093250489E396E06BEDB2
:1037F00073E02FC086E18093250489E396E064EAB4
:1038000073E027C087E18093250489E396E06AE5A9
:1038100073E01FC088E18093250489E396E069E4A2
:1038200073E017C089E18093250489E396E065E39E
:1038300073E00FC08AE18093250489E396E060E29B
:1038400073E007C08BE18093250489E396E068EF7D
:1038500072E00E94B82B34C089E396E06EED72E00E
:103860000E94B82B8091C30391E01DC089E396E0CC
:1038700068EC72E00E94B82B8091C30392E013C001
:1038800089E396E063EB72E00E94B82B8091C3035A
:1038900094E009C089E396E068E972E00E94B82BE1
:1038A0008091C30398E089278093C3038FEF8093AF
:1038B00025040E94751A04C089E396E00E94AD2E8B
:1038C00089E396E00E94732E892BB1F762C1822FA3
:1038D0000E94D416882309F45CC180918B0488234C
:1038E00021F48FEF809325044CC186E294E060E0E0
:1038F00070E040E050E00E94A2069B01AC016091A4
:103900002504862F992787FD9095A92FB92FFC01B3
:103910003197EB31F10508F024C1ED55FF4F0C94C0
:103920002030E62FFF27E7FDF0958091220490E0FC
:103930008E179F070CF415C1DA01C9010197A1097F
:10394000B1098097A105B10548F0A8E2FA2E00E080
:1039500010E06F010894C108D10825C0EB54FC4F5A
:10396000822F81508083E5C0612F70E0660F771F42
:103970006F5F7B4FFB01808190E08C159D0591F47A
:103980008F2D90E0A0E0B0E082179307A407B50761
:1039900041F4F601EB54FC4FDB0111968C918183CD
:1039A00001E0F3941F5F809121041817E8F2BFC073
:1039B0002F3F31054105510511F008F0D2C0209389
:1039C000CD03B7C02F3F31054105510511F008F077
:1039D000C8C02093CE03ADC02F3F3105410551052E
:1039E00011F008F0BEC02093CF03A3C0809126043D
:1039F0008062803719F587E294E060E070E040E093
:103A000050E00E94A2069B01AC01DC01CB010197B2
:103A1000A109B1090897A105B10508F0B5C0CA010F
:103A2000B90124ED30E340E050E00E947A2F9B0181
:103A3000AC012A5E3C4A4A46554E24C0863611F5F2
:103A400087E294E060E070E040E050E00E94A2066F
:103A50009B01AC01DC01CB010197A109B1090797DA
:103A6000A105B10508F090C0CA01B90128EA31E604
:103A700040E050E00E947A2F9B01AC01245E3C4361
:103A80004E46544E211531054105510561F0DA01CC
:103A9000C9018054914EAD49B8418158904FAA4F09
:103AA000B24008F05EC02093C5033093C603409334
:103AB000C7035093C8033DC02F3F31054105510551
:103AC00011F008F04EC02093C90333C0DA01C901D8
:103AD0000197A109B1098F3F9105A105B10508F032
:103AE00040C02093CA0325C0DA01C901845C994013
:103AF000A040B0408D549D41A040B04030F4309380
:103B0000CC032093CB0301E001C000E02115310577
:103B10004105510511F48FEF07C0213431054105EE
:103B2000510528F4822F81508093C40302C00023E2
:103B3000C1F080918C048823D1F48091D9039091B5
:103B4000DA03A091DB03B091DC030196A11DB11D46
:103B50008093D9039093DA03A093DB03B093DC0343
:103B600006C089E396E068EA71E00E942E2D0E946B
:103B7000CA168FEF8093250489E396E06AE00E94DD
:103B8000CC2B0E94751A05C021E030E040E050E0E7
:103B90007ECF6C96E8E00C940F3089E396E06CE4FD
:103BA00072E00E94B82B89E396E064E372E00E9421
:103BB000B82B89E396E00E94732E892B31F089E3BC
:103BC00096E00E94AD2E0E94201B0E94F4148230C9
:103BD00019F0833069F405C089E396E066E172E08C
:103BE00004C089E396E06FEF71E00E94B82B08955E
:103BF0008FEF8093250410928C040E94751A0CC0DC
:103C000089E396E00E94732E892B31F089E396E0D8
:103C10000E94AD2E0E94201B809125048E3F81F7CB
:103C2000089580912504992787FD9095A92FB92F94
:103C3000FC013196EB30F10508F074C0E254FF4FFF
:103C40000C94203089E396E064E678E00E94B82B7B
:103C500083E793E00E94441A89E396E06CE478E0FD
:103C60000E94B82B89E396E067E278E00E94B82BC7
:103C700089E396E06DEF77E00E94B82B89E396E048
:103C80006CED77E00E94B82B89E396E06FEA77E06D
:103C90000E94B82B89E396E069E877E00E94B82B90
:103CA00089E396E065E677E00E94B82B89E396E029
:103CB0006EE377E00E94B82B89E396E00E94A22B86
:103CC0000E941D192FC089E396E061E277E028C0C9
:103CD00089E396E06CEF76E023C089E396E067EE37
:103CE00076E01EC089E396E068EC76E019C089E3CF
:103CF00096E064E876E014C089E396E06FE676E04B
:103D00000FC089E396E06AE576E00E94B82B89E36C
:103D100096E064E176E004C089E396E06EEF75E03A
:103D20000E94B82B6AE070E080E090E00E94052AD3
:103D300004C089E396E00E94AD2E89E396E00E94DC
:103D4000732E892BB1F70895A2E2B0E0EAEAFEE112
:103D50000C94E92F8E010F5F1F4F80E1D8011D9257
:103D60008A95E9F789E396E066EC71E00E942E2DD2
:103D70000E94A01520E431EE4DE958E12F8F38A3C1
:103D800049A35AA380EC91EDA8E9BBE18B8F9C8FEE
:103D9000AD8FBE8F24EF31E040E050E02F8B388FA5
:103DA000498F5A8F30E5C32E33ECD32EE12CF12C02
:103DB00020E4422E21EE522E2DE9622E28E1722EB1
:103DC00088249924540133241E8A1D8A198A1A8A48
:103DD0001B8A1C8AFFC089E396E00E94AD2E8434C2
:103DE000B9F0853430F48332B9F18C3209F0CCC0AB
:103DF00044C0833509F0C8C02F8D38A149A15AA10C
:103E0000C901DA012C013D01882499245401E2C042
:103E100089E396E064E40E949A2B89E396E040E40B
:103E200051EE6DE978E12AE030E00E94CE2C89E382
:103E300096E06CE20E949A2B89E396E040EC51ED0B
:103E400068E97BE12AE030E00E94CE2C89E396E02D
:103E50006CE20E94CC2BBEC019821A821B821C828B
:103E60001D821E821F82188619861A861B861C8652
:103E70001D861E861F86188A3AC0339434E0331696
:103E800009F0A8C069817A818B819C8128EE33E09A
:103E900040E050E00E947A2F6F8F78A389A39AA305
:103EA0006D817E818F8198850E947A2F6B8F7C8FA8
:103EB0008D8F9E8F89859A85AB85BC858F8B988FDA
:103EC000A98FBA8F6D857E858F8598890E947A2FFC
:103ED0006B017C0190E2C9169EE4D90690E0E906E8
:103EE00090E0F90630F48CE162E30E94C00A3324CA
:103EF00071C0A0E3CA16A5E7DA06A0E0EA06A0E0D2
:103F0000FA0618F48CE162E2F0CFB0E4CB16BCE91B
:103F1000DB06B0E0EB06B0E0FB0618F48CE166E2ED
:103F2000E4CFE0E5CE16E3ECDE06E0E0EE06E0E00E
:103F3000FE0618F48CE162E1D8CFF0E6CF16FAEE77
:103F4000DF06F0E0EF06F0E0FF0618F48CE165E133
:103F5000CCCF20E7C21621E1D20621E0E20620E024
:103F6000F20618F48CE161E0C0CF30EAC31636E8FF
:103F7000D30631E0E30630E0F30618F48CE163E0A9
:103F8000B4CF8CE165E0B1CF90ED292E280E49E049
:103F9000421500F1032D10E0000F111F000F111F3B
:103FA00081E090E08C0F9D1F080F191FD8016D91C3
:103FB0007D918D919C912AE030E040E050E00E949C
:103FC0007A2F620D711D811D911DF801608371832F
:103FD0008283938389E396E00E94732E892B09F0F4
:103FE000FACE81149104A104B10489F4C301B20191
:103FF0000E94360B61E070E080E090E00E94052AAC
:10400000FFEFFE8B1D8A198A1A8A1B8A1C8A2F8948
:10401000388D498D5A8D82169306A406B506E0F4B4
:104020000E94E10A29893A894B895C89280F311D50
:10403000411D511D298B3A8B4B8B5C8B3D89381769
:1040400008F48D8B4E89841708F48E8B0894811C9C
:10405000911CA11CB11C56C0C301B20128EE33E073
:1040600040E050E00E94AC2F89E396E0BA01A9013C
:104070002AE030E00E94602C89E396E06CE20E9426
:104080009A2B89E396E06D894AE050E00E94A82CC3
:1040900089E396E06CE20E949A2B69897A898B8980
:1040A0009C89A50194010E94AC2F89E396E0BA0196
:1040B000A9012AE030E00E94602C89E396E06CE2DE
:1040C0000E949A2B89E396E06E894AE050E00E94B4
:1040D000A82C89E396E06CE20E94CC2B4C0C5D1C72
:1040E0006E1C7F1C8B8D9C8DAD8DBE8D84159505B2
:1040F000A605B70520F44F8C58A069A07AA08824A3
:10410000992454012F8D38A149A15AA1285E33402A
:104110004040504009F05ECFA296E2E10C94053099
:10412000A0E0B0E0E6E9F0E20C94F42F0E94DF2971
:104130006115710581059105C9F30E9499061092D8
:10414000D9031092DA031092DB031092DC03DD2412
:10415000E090D903F090DA030091DB031091DC03C7
:10416000102F0F2DFE2CEE240E9494062FEF30E02E
:1041700040E050E00E94CE2FE60EF71E081F191FE8
:10418000E092D903F092DA030093DB031093DC038F
:10419000D39444E0D416E1F6CFEDD3E000E010E094
:1041A00040E1E42E47E2F42E4EC00F5F19F40E9466
:1041B0004D084DC00E94940622E330E040E050E0FC
:1041C0000E94CE2F6F5FEFEDF3E090E004C081918D
:1041D000861759F39F5F9117D0F38091DE0390E02B
:1041E0008E9D90018F9D300D9E9D300D1124862F48
:1041F00090E0AC01249FC001259F900D349F900D4D
:104200001124AA2797FDA095BA2F2091D5033091AC
:10421000D6034091D7035091D803820F931FA41F58
:10422000B51F20919D0330919E0340919F035091B3
:10423000A003281739074A075B0708F4B6CF69932C
:104240001F5F183121F08881882309F0AECFCDB7E8
:10425000DEB7E7E00C94103080E060E00E94F915D2
:10426000882331F081E060E00E94F915882341F451
:104270000E9492080E944D080E9490200E949F1662
:104280000895AAE5B0E0E7E4F1E20C94F52F8B0184
:104290007A018B3009F425C18C3040F5853009F462
:1042A00084C0863080F4823009F459C0833020F411
:1042B000813009F04FC242C0833009F461C08430BC
:1042C00009F048C265C0883009F49DC0893038F4CF
:1042D000863009F486C0873009F03CC28CC0893032
:1042E00009F499C08A3009F035C2C9C0893609F489
:1042F00081C18A3680F4863609F42CC1873620F4D1
:10430000853609F027C20DC1873609F43CC18836CD
:1043100009F020C240C18C3609F4C3C18D3638F48F
:104320008A3609F472C18B3609F014C2AEC18D36DB
:1043300009F4EBC1873C09F00DC2FFC181E069E2DD
:1043400070E00E94851100ED13E0F80181918F016A
:104350000E946E11F3E0093F1F07B9F703C282E024
:104360006BE170E00E94851105EB13E0F80181918B
:104370008F010E946E11F3E0003D1F07B9F7F2C1F3
:1043800083E061E070E00E9485110E94F414E8C1AE
:1043900084E061E070E00E94851181E00E946E116E
:1043A0000E9467110E94A41EDFC16091210470E089
:1043B000660F771F85E00E94851100E010E008C0BD
:1043C000F801EF5FFB4F80810E946E110F5F1F4F5E
:1043D0008091210490E0880F991F0817190780F336
:1043E000C1C186E062E070E00E94851183E793E03E
:1043F0000E947C11B7C187E061E070E00E948511E6
:1044000080912204ADC188E061E070E00E948511D6
:1044100080919B03A5C186E68983CE01019661E068
:104420000E94CD0F0E94840C83E080939A0368EC75
:1044300070E080E090E00E94052A80919A03843029
:10444000E1F48FE70E94960A0E94AA0A89838634C3
:1044500071F489E060E270E00E94851110E00E9432
:10446000AA0A0E946E111F5F1032C9F77BC189E052
:1044700061E070E00E948511C6C089E06CC18AE0ED
:1044800069E170E00E94851110929C038091A30560
:10449000882351F08091A1039091A203A091A303DE
:1044A000B091A403806809C08091A1039091A203F8
:1044B000A091A303B091A4038F778093A10390935D
:1044C000A203A093A303B093A4030CE913E0F801A3
:1044D00081918F010E946E11F3E0053B1F07B9F730
:1044E00041C18BE061E270E00E9485118091C004BF
:1044F0008F3F39F08091C0048F5F8093C00481505A
:1045000002C08091C0040E946E1110E0812F0E94B1
:10451000A4110E94190A0E947C111F5F1031B1F78B
:1045200021C185E661E070E00E9485110932110524
:1045300009F015C120E030E0F901E053FC4FD7014C
:10454000A20FB31F8C9180832F5F3F4F293231051B
:1045500099F759C086E661E070E00E9485110B3141
:10456000110509F0FCC020E030E0F901EB54FC4FEC
:10457000D701A20FB31F8C9180832F5F3F4F2B3148
:10458000310599F740C087E661E070E00E9485112F
:104590000E949F1638C088E661E070E00E94851195
:1045A00085E78A83DE011396E5EBF3E08BE101906A
:1045B0000D928150E1F7CE0102966CE10E94CD0F81
:1045C0000E94840C83E080939A0360E273E080E0B1
:1045D00090E00E94052A80919A03843009F0BFC0C0
:1045E0008FE70E94960A0E94AA0A8A83853509F0FD
:1045F000B6C009C089E661E070E00E9485110E94A2
:104600004D080E94920881E0ABC08AE661E070E04C
:104610000E94851189E68E8FCE014E9661E00E9440
:10462000CD0F0E94840C83E080939A0360E273E0D4
:1046300080E090E00E94052A80919A03843009F07E
:104640008EC08FE70E94960A0E94AA0A8E8F8E0162
:10465000015E1F4F6AE3E62EF12CEC0EFD1E0E9458
:10466000AA0AF80181938F01EE15FF05C1F7A5EBAA
:10467000B3E0FE017F968BE101900D928150E1F74E
:104680008E8D893409F06BC0BECF8BE661E070E09F
:104690000E948511F70180810E94BA160E942C2188
:1046A000B2CF8CE661E070E00E9485110032110506
:1046B00071F487E68AAFDE01DB96F70180E20190B4
:1046C0000D928150E1F7CE01CA9661E205C087E400
:1046D0008AAFCE01CA9661E00E94CD0F0E94840C81
:1046E00083E080939A036CE474E080E090E00E94A1
:1046F000052A80919A03843091F58FE70E94960AEB
:104700000E94AA0A873459F57ECF8DE661E070E0F9
:104710000E9485110931110511F520E030E0F90101
:10472000E456FC4FD701A20FB31F8C9180832F5FFB
:104730003F4F2931310599F766CF87EC61E070E092
:104740000E94851181E00E946E110E9467111092F3
:10475000FF030AC08AEC61E070E00E94851180E0EE
:104760000E946E110E946711C65ADF4FE6E00C945A
:104770001130A0E0B0E0EFEBF3E20C94F12F84E015
:10478000A82E06E0B02E15E0C12E07E315E0B4E632
:10479000DB2EA2E0EA2EF3E0FF2EA1C089E396E033
:1047A0000E94AD2E982F8093A2058091A1058330A1
:1047B00021F1843028F4813099F08230B8F409C0B6
:1047C000853009F448C0853020F1863009F087C073
:1047D0005FC0953B09F083C081E08093A1057FC055
:1047E000923609F07AC0E092A10579C09093A005B5
:1047F00090939F05F092A10572C090939D05109231
:104800009E0580919F05892780939F05A092A10511
:1048100066C0D92FC0E020919D0530919E052C2BBC
:104820003D2B30939E0520939D0580919F05892700
:1048300080939F05C092A1052536310508F44FC02D
:104840008CEC61E070E00E94851181E00E946E11A5
:104850000E94671142C020919B0530919C05F9018F
:10486000E95CFA4F908380919F05892780939F058B
:104870002F5F3F4F30939C0520939B0580919D05B2
:1048800090919E052817390750F1B092A10527C0D5
:1048900080919F05891759F460919B0570919C0543
:1048A0008091A00547E355E00E9441210DC08BECAB
:1048B00062E070E00E9485118091A0050E946E1157
:1048C000809100040E946E11F8018D2D11928A953D
:1048D000E9F710929C0510929B051092A10589E3BF
:1048E00096E00E94732E892B09F058CFCDB7DEB722
:1048F000EAE00C940D3081E08093FF0308C089E367
:1049000096E00E94732E892B11F00E94B9238091AA
:10491000FF038823A1F708951F93109125041F3FDB
:1049200009F0F1C0893409F467C08A3428F5883366
:1049300009F479C0893368F4803309F486C081337F
:1049400008F06FC08B3109F44DC0813209F0D5C039
:104950003DC0813409F49AC0823438F4893309F4B3
:1049600072C0803409F0C9C031C0823409F4A1C0DA
:10497000863409F0C2C052C0823609F49AC0833628
:1049800090F4883579F1893538F4823509F43FC0DF
:10499000833509F0B2C01FC08A3509F4A9C0813639
:1049A00009F0ABC073C0823791F1833730F486369B
:1049B000A9F1893609F0A1C01FC0883799F08A375C
:1049C00009F496C0833709F098C005C089E396E0E2
:1049D00069E471E019C00E949F1689E396E063EDD7
:1049E00071E006C00E942C2189E396E06DEE71E033
:1049F0000E942E2D8EEF7FC00E944D080E949208CB
:104A000089E396E06CE072E00E942E2D76C00E9451
:104A1000902089E396E065E272E0F6CF0E943D17B0
:104A20006CC0805368C089E396E06CEE71E00E9430
:104A3000B82B9091F803892F885F8871977E892B16
:104A40008093F80320C089E056C089E396E069EDC1
:104A500071E00E94B82B8091A1039091A203A091D4
:104A6000A303B091A40320E130E040E050E08227AE
:104A70009327A427B5278093A1039093A203A09323
:104A8000A303B093A4031093250437C089E396E0F1
:104A900063EC71E00E94B82B8091A1039091A20376
:104AA000A091A303B091A40320E430E040E050E0E3
:104AB00012C089E396E062EB71E00E94B82B80910E
:104AC000A1039091A203A091A303B091A40320E2BB
:104AD00030E040E050E082279327A427B527809359
:104AE000A1039093A203A093A303B093A40302C0D5
:104AF0000E94CD1D8FEF80932504809125048E3F69
:104B000009F4DDC0D4C00E94D416882309F4D7C0AC
:104B100080918B04882321F48FEF80932504C7C0F4
:104B200086E294E060E070E040E050E00E94A2067F
:104B30009B01AC0180912504992787FD9095A92FB1
:104B4000B92FFC013197E930F10508F08CC0E7532B
:104B5000FF4F0C942030DA01C9018154914EAD49C8
:104B6000B8418F57904FAA4FB24008F07CC02093B5
:104B7000D5033093D6034093D7035093D8039AC0FC
:104B80002093D9033093DA034093DB035093DC0383
:104B900081E080938C048EC0283031054105510599
:104BA00008F061C02093DD0385C0DA01C9010197D7
:104BB000A109B1090A97A105B10508F054C02093D5
:104BC000DE0378C086E294E06DE371E00E94BE07E8
:104BD00010E00EC0183130F4E12FF0E0E053FC4F4C
:104BE00087871F5F80E090E06DE371E00E94BE0761
:104BF000009759F00E94A007009761F706C0E12FC7
:104C0000F0E0E053FC4F17861F5F1831C0F352C02D
:104C1000253031054105510530F52093F7034AC091
:104C2000DA01C9010197A109B1090697A105B105EA
:104C3000D0F48091F803887F822B8093F8033AC0E8
:104C4000DA01C9010197A109B1098050924CA14034
:104C5000B04048F42093D1033093D2034093D30360
:104C60005093D40327C089E396E068EA71E00E947C
:104C70002E2D13C08091D9039091DA03A091DB030C
:104C8000B091DC030196A11DB11D8093D9039093CF
:104C9000DA03A093DB03B093DC030E94CA168FEF04
:104CA0008093250489E396E06AE00E94CC2B0E9461
:104CB000111E05C080918C048823E1F2EECF1F9174
:104CC00008958FEF8093250410928C040E94111E8A
:104CD0000CC089E396E00E94732E892B31F089E3A2
:104CE00096E00E94AD2E0E948C24809125048E3F78
:104CF00081F76AE070E080E090E00E94052A04C03D
:104D000089E396E00E94AD2E89E396E00E94732E1F
:104D1000892BB1F70895AAE2B0E0E1E9F6E20C943C
:104D2000EE2F0E94D1297B018C0181E00E94A50B0E
:104D300004C089E396E00E94AD2E89E396E00E94CC
:104D4000732E892BB1F75E984098DD24D39432E618
:104D5000732E22E0822E912C8C0E9D1E5E010894F3
:104D6000A11CB11C93E0C92E0E94D12920E030E0A3
:104D70006E197F09800B910B693C710581059105C6
:104D800010F021E030E08D2D90E028233923232BF3
:104D9000A9F10E94D1297B018C015D9A419A80ED95
:104DA00097E00E94DA117982D401E0EDF3E089E224
:104DB00001900D928150E1F7C5016AE20E94CD0F8A
:104DC0005D98419880E090E00E94DA11C0929A03C9
:104DD0000E94840C62E370E080E090E00E94052A6B
:104DE00080919A03843051F4C0929A038FE70E9415
:104DF000960A0E94AA0A823409F4DD2483E10E9403
:104E0000032B892B69F5DD24D3942AC05E9A409A3E
:104E10005D9A419A89E396E00E94AD2E8D3091050E
:104E200069F08E3091051CF40A97B1F407C0833203
:104E3000910569F08234910579F40CC089E396E01C
:104E400064EA71E00E94B82B0E94612605C00E94AE
:104E5000A41E02C00E947B245E9840985D984198F1
:104E600089E396E00E94732E892B09F47DCFCECF83
:104E70008F929F92AF92BF92CF92DF92EF92FF926A
:104E80000F931F9383E10E94032B892B09F083C0AA
:104E900068EC70E080E090E00E94052A80E090E0FD
:104EA0000E94DA110E94D1295B016C0140ECE42ED2
:104EB00042E1F42E012D112DE60EF71E081F191FD9
:104EC00006C083E10E94032B892B09F062C00E9477
:104ED000D1296E157F058007910798F383E10E9421
:104EE000032B892B09F055C080ED97E00E94DA1161
:104EF0000E94D1297B018C0199249394882488E411
:104F000096E2A0E0B0E0A80EB91ECA1EDB1E29C0C2
:104F1000AE14BF04C006D10638F480ED97E00E94BD
:104F2000DA11882483941DC00E94D1296E197F094B
:104F3000800B910B693C71058105910590F00E94F1
:104F4000D1297B018C0180E0992009F481E0982E21
:104F5000882319F480E090E002C080ED97E00E9481
:104F6000DA1183E10E94032B892B91F280E090E01B
:104F70000E94DA11882049F080919B038F5F837033
:104F80000E94BA160E942C2106C00E9490200E9406
:104F90009F160E948B261F910F91FF90EF90DF903C
:104FA000CF90BF90AF909F908F90089580E06DEF6D
:104FB00077E042E050E00E940C290895EF92FF92C2
:104FC0000F931F9380E00E9419080E94C51186E08C
:104FD00061E00E94642A85E061E00E94642A8EE01C
:104FE00061E00E94642A8FE061E00E94642A83E10C
:104FF00060E00E94642A88E060E00E94642A88E001
:1050000061E00E94D02A0E94CC1489E396E040E03F
:1050100052EC61E070E00E94EC2D0E94AD160E94FF
:105020002C210E94640D8FEF8093C0040E94D6272C
:1050300078940E94D1297B018C018091C0048F3F1C
:1050400009F0DFC00E94D1296E197F09800B910BF6
:10505000605D77408040904008F0D3C0EECF89E398
:1050600096E00E94AD2E89E396E00E94732E892B74
:10507000B1F789E396E062E472E00E942B2D83E7AA
:1050800093E00E94441A89E396E069E572E00E9489
:105090002B2D89E396E067E070E04AE050E00E9443
:1050A000172D62E370E080E090E00E94052A89E31A
:1050B00096E00E94732E04970CF189E396E00E941B
:1050C000AD2E82349105D1F489E396E00E94AD2E95
:1050D0008E34910599F489E396E00E94AD2E8434D4
:1050E000910561F489E396E00E94AD2E819731F439
:1050F00080E090E00E94DA110E948B264091D1035B
:105100005091D2036091D3037091D403DB01CA01A3
:105110000197A109B1090497A105B10568F440936D
:10512000C104433029F040E052EC61E070E004C07B
:1051300040EA56E861E070E089E396E00E94EC2DD9
:105140000E9438275E98409880E090E00E94DA1133
:105150000E94640D1092A5048091A10383FF11C0E9
:105160008091E503882351F08091EC03882331F08E
:105170008091F303882311F087E001C085E08093DC
:10518000A50480E00E94A50B8091A4040E94CB0A94
:105190000E94840C10922B0510922C0510922D0564
:1051A00010E015C062E370E080E090E00E94052A04
:1051B00080ED97E00E94DA1162E370E080E090E019
:1051C0000E94052A80E090E00E94DA111F5F809122
:1051D0009B03811738F78091F80390E084FF09C0A2
:1051E00020E088719070489709F421E0822F0E9496
:1051F000D5148FE00E9419081F910F91FF90EF9036
:10520000089580ED97E00E94DA1183E161E00E9449
:10521000D02A5E9A409A27CF823000F5E82FF0E03E
:10522000EE0FFF1FEC55FA4F71836083882319F04E
:105230008130A1F408C0809169008C7F842B809319
:105240006900E89A089580916900440F551F440F42
:10525000551F837F842B80936900E99A08951F92DC
:105260000F920FB60F9211242F933F934F935F939A
:105270006F937F938F939F93AF93BF93EF93FF931E
:105280008091A4059091A505892B29F0E091A405B2
:10529000F091A5050995FF91EF91BF91AF919F9175
:1052A0008F917F916F915F914F913F912F910F90CF
:1052B0000FBE0F901F9018951F920F920FB60F926E
:1052C00011242F933F934F935F936F937F938F930B
:1052D0009F93AF93BF93EF93FF938091A605909117
:1052E000A705892B29F0E091A605F091A70509955E
:1052F000FF91EF91BF91AF919F918F917F916F91AE
:105300005F914F913F912F910F900FBE0F901F9083
:1053100018951F920F920FB60F9211242F933F935F
:105320008F939F93AF93BF938091AC059091AD0500
:10533000A091AE05B091AF053091B0050196A11DC9
:10534000B11D232F2D5F2D3720F02D570196A11D64
:10535000B11D2093B0058093AC059093AD05A0934B
:10536000AE05B093AF058091A8059091A905A091D5
:10537000AA05B091AB050196A11DB11D8093A805AA
:105380009093A905A093AA05B093AB05BF91AF91E7
:105390009F918F913F912F910F900FBE0F901F9073
:1053A00018958FB7F8942091AC053091AD054091D8
:1053B000AE055091AF058FBFB901CA0108959FB7DF
:1053C000F8942091A8053091A9054091AA05509123
:1053D000AB0586B5A89B06C08F3F21F02F5F3F4FDE
:1053E0004F4F5F4F9FBF542F432F322F2227280F3D
:1053F000311D411D511D82E0220F331F441F551FD7
:105400008A95D1F7B901CA010895EF92FF920F93DF
:105410001F93CF93DF937B018C010E94DF29EB0167
:105420000EC00E94DF296C1B7D0B685E7340C8F3C1
:105430000894E108F10801091109C851DC4FE11491
:10544000F1040105110569F7CDB7DEB7E6E00C946C
:105450001130789484B5826084BD84B5816084BD48
:1054600085B5826085BD85B5816085BDEEE6F0E0DD
:10547000808181608083E1E8F0E010828081826039
:105480008083808181608083E0E8F0E080818160BA
:105490008083E1EBF0E0808184608083E0EBF0E0EA
:1054A000808181608083EAE7F0E08081846080838E
:1054B0008081826080838081816080838081806838
:1054C00080831092C1000895CF93DF93482F50E05E
:1054D000CA018D5F934FFC0134914151544FFA0141
:1054E0008491882369F190E0880F991FFC01EF52A5
:1054F000F44FA591B491FC01E552F44FC591D491BC
:10550000662351F42FB7F8948C91932F90958923AB
:105510008C93888189230BC0623061F42FB7F89493
:105520008C91932F909589238C938881832B8883EA
:105530002FBF06C09FB7F8948C91832B8C939FBF8D
:10554000DF91CF910895833071F0843028F4813059
:10555000A1F0823021F514C08630B1F08730D1F04F
:105560008430E9F404C0809180008F7703C080917B
:1055700080008F7D80938000089584B58F7702C06E
:1055800084B58F7D84BD08958091B0008F7780931E
:10559000B00008958091B0008F7D8093B000089591
:1055A000FF920F931F93F62E482F50E0CA01895E99
:1055B000934FFC012491CA018D5F934FFC0114911C
:1055C0004151544FFA0104910023C9F0222319F0EC
:1055D000822F0E94A32AE02FF0E0EE0FFF1FE5527A
:1055E000F44FA591B4919FB7F894FF2021F48C91CA
:1055F0001095812302C08C91812B8C939FBF1F91AA
:105600000F91FF9008950F931F93482F50E0CA0108
:10561000895E934FFC012491CA018D5F934FFC0179
:1056200004914151544FFA011491112319F420E0CF
:1056300030E015C0222319F0822F0E94A32A812F67
:1056400090E0880F991F8B51944FFC01A591B49164
:105650008C9120E030E0802311F021E030E0C9019E
:105660001F910F910895982F8E3008F09E509770DB
:10567000809148038295880F880F807C892B8093C6
:105680007C0080917A00806480937A0080917A0017
:1056900086FDFCCF2091780040917900942F80E026
:1056A00030E0282B392BC9010895A0E0B0E0EBE5EC
:1056B000FBE20C94F32F7C016B018A01C0E0D0E087
:1056C0000FC0D6016D916D01D701ED91FC91019054
:1056D000F081E02DC7010995C80FD91F0150104076
:1056E0000115110571F7CE01CDB7DEB7E8E00C94D6
:1056F0000F30EF92FF920F931F93CF93DF937C01B4
:105700008B01C0E0D0E0F8010F5F1F4F649166236A
:1057100059F0D701ED91FC910190F081E02DC70186
:105720000995C80FD91FEFCFCE01CDB7DEB7E6E0A0
:105730000C941130DC01ED91FC910190F081E02D91
:1057400009950895EF92FF920F931F938C016DE0DE
:105750000E949A2B7C01C8016AE00E949A2B9C014E
:105760002E0D3F1DC9011F910F91FF90EF900895DD
:10577000EF92FF920F931F937C010E94792B8C0173
:10578000C7010E94A22B9C01200F311FC9011F914C
:105790000F91FF90EF900895EF92FF920F931F9358
:1057A0007C010E949A2B8C01C7010E94A22B9C01B4
:1057B000200F311FC9011F910F91FF90EF900895A5
:1057C000CF93DF93EC016115710519F420E030E00F
:1057D0000FC0DB010D900020E9F71197A61BB70B56
:1057E000E881F9810280F381E02DAD0109959C01EA
:1057F000C901DF91CF9108954F925F927F928F926E
:105800009F92AF92BF92CF92DF92EF92FF920F934F
:105810001F93DF93CF93CDB7DEB7A1970FB6F89460
:10582000DEBF0FBECDBF2C01742ECB01223008F499
:105830002AE019A231E2C32ED12CCC0EDD1E822E1D
:105840009924AA24BB24672D752FA50194010E94D9
:10585000AC2F79018A01C801B701A50194010E940A
:105860007A2F472D461B0894C108D1084A3010F4FE
:10587000405D01C0495CF6014083E114F10401057B
:10588000110521F07E2C5F2DC801DDCFC201B601CC
:105890000E94E02BA1960FB6F894DEBF0FBECDBFDD
:1058A000CF91DF911F910F91FF90EF90DF90CF90FC
:1058B000BF90AF909F908F907F905F904F90089592
:1058C000DC012115310541F4ED91FC910190F0814D
:1058D000E02D642F099508950E94FC2B0895EF9206
:1058E000FF920F931F937C010E94602C8C01C701D3
:1058F0000E94A22B9C01200F311FC9011F910F9103
:10590000FF90EF900895EF92FF920F931F939A01EB
:105910007B0100E010E0B801A7010E94602C1F91FC
:105920000F91FF90EF900895EF92FF920F931F93C6
:105930007C010E94832C8C01C7010E94A22B9C0138
:10594000200F311FC9011F910F91FF90EF90089513
:10595000EF92FF920F931F939A01E62EFF2400E02F
:1059600010E0B801A7010E94602C1F910F91FF90D9
:10597000EF900895EF92FF920F931F937C010E9486
:10598000A82C8C01C7010E94A22B9C01200F311F63
:10599000C9011F910F91FF90EF900895A0E0B0E032
:1059A000E4EDFCE20C94F32FEC016A017B0121157C
:1059B000310541F4E881F9810190F081E02D642FF7
:1059C00009951BC02A303105B1F477FF13C06DE291
:1059D0000E949A2B8C0144275527BA014C195D0966
:1059E0006E097F09CE012AE00E94FC2B9C01200F4A
:1059F000311F04C02AE00E94FC2B9C01C901CDB7D5
:105A0000DEB7E8E00C940F30EF92FF920F931F93F4
:105A10007B019A010027F7FC0095102FB801A70120
:105A20000E94CE2C1F910F91FF90EF900895EF925E
:105A3000FF920F931F937C010E94042D8C01C701DC
:105A40000E94A22B9C01200F311FC9011F910F91B1
:105A5000FF90EF9008950E94E02B0895EF92FF923F
:105A60000F931F937C010E942B2D8C01C7010E9474
:105A7000A22B9C01200F311FC9011F910F91FF9094
:105A8000EF90089508951F920F920FB60F92112470
:105A90002F933F934F938F939F93EF93FF93809117
:105AA000C00082FD1DC04091C6002091F1053091DB
:105AB000F2052F5F3F4F2F7330708091F305909167
:105AC000F4052817390771F0E091F105F091F2051E
:105AD000EF54FA4F40833093F2052093F10502C052
:105AE0008091C600FF91EF919F918F914F913F91CF
:105AF0002F910F900FBE0F901F9018951F920F922D
:105B00000FB60F9211242F933F938F939F93EF9390
:105B1000FF9320913506309136068091370690919B
:105B200038062817390731F48091C1008F7D8093A2
:105B3000C10014C0E0913706F0913806EB50FA4FDF
:105B40002081809137069091380601968F7390706E
:105B500090933806809337062093C600FF91EF910B
:105B60009F918F913F912F910F900FBE0F901F909B
:105B70001895A0E0B0E0EFEBFDE20C94EF2FFC01F4
:105B80001382128288EE93E0A0E0B0E084839583D4
:105B9000A683B7838BE893E09183808375876487BE
:105BA00057874687318B208B138B028BF58AE48ACB
:105BB000D78AC68AB18EA08E938E828E8F85848F6F
:105BC0008889858F8989868F8A89878F8B8980A329
:105BD0002096ECE00C940B30AF92BF92DF92EF92E4
:105BE000FF920F931F93CF93DF93EC017A018B0108
:105BF000DD24403081EE580780E0680780E07807B8
:105C000011F0DD24D39491E0A92EB12CEC89FD890B
:105C1000DD2069F0C50108A002C0880F991F0A9411
:105C2000E2F7808360E079E08DE390E005C01082C8
:105C300060E874E88EE190E0A80197010E94AC2F23
:105C40002150304040405040569547953795279514
:105C500080E12030380720F0DD2011F0DD24D6CFA0
:105C6000E889F9893083EA89FB89208319A2EE89C2
:105C7000FF89408121E030E0C9010C8C02C0880F0F
:105C8000991F0A94E2F7482B4083EE89FF894081EF
:105C9000C9010D8C02C0880F991F0A94E2F7482BA6
:105CA0004083EE89FF894081C9010E8C02C0880FB4
:105CB000991F0A94E2F7482B4083EE89FF8980817F
:105CC0000F8C02C0220F331F0A94E2F7209528237D
:105CD0002083DF91CF911F910F91FF90EF90DF9084
:105CE000BF90AF900895DC011C96ED91FC911D973B
:105CF000E05CFF4F2191319180819181281B390B0C
:105D00002F733070C901089589E396E00E94732EC5
:105D1000892B11F00E94422D0895DC011C96ED9113
:105D2000FC911D97E05CFF4F20813181E054F040F1
:105D3000DF01AE5BBF4F8D919C91119728173907FA
:105D400019F42FEF3FEF07C08D919C91E80FF91FD9
:105D50008081282F30E0C9010895DC011C96ED9167
:105D6000FC911D97E05CFF4F20813181E054F040B1
:105D7000DF01AE5BBF4F8D919C91119728173907BA
:105D800019F42FEF3FEF10C08D919C911197E80F00
:105D9000F91F20818D919C91119701968F739070BE
:105DA00011969C938E9330E0C9010895DC01919681
:105DB0008C919197882339F05496ED91FC915597E9
:105DC000808186FFF9CF91961C920895CF93DF933F
:105DD000EC01EE85FF85E05CFF4F20813181E054CE
:105DE000F0402F5F3F4F2F733070DF01AE5BBF4F2E
:105DF0008D919C91119728173907D1F3E05CFF4FE3
:105E000080819181E054F040E80FF91F6083EE85B6
:105E1000FF85E05CFF4F31832083EE89FF8920817D
:105E200081E090E00F8C02C0880F991F0A94E2F77E
:105E3000282B208381E089A3EC89FD8980818064FF
:105E4000808381E090E0DF91CF9108958F929F92BF
:105E5000AF92BF92CF92DF92EF92FF920F931F9378
:105E600000D000D00F92EDB7FEB7319684E0ADB709
:105E7000BEB711968C9383E0818387E0828385E0AF
:105E8000838381E0848389E396E061EB75E045EFED
:105E900055E025EC30E004EC10E0B0ECEB2EF12CFA
:105EA000A1ECCA2ED12CF2ECAF2EB12CE6EC8E2E4A
:105EB000912C0E94B92D0F900F900F900F900F9082
:105EC0001F910F91FF90EF90DF90CF90BF90AF9018
:105ED0009F908F900895CF93DF930E94292A0E946C
:105EE000DE27C4E8DEE20E94E4112097E1F30E947D
:105EF000842EF9CF629FD001739FF001829FE00D45
:105F0000F11D649FE00DF11D929FF00D839FF00D38
:105F1000749FF00D659FF00D9927729FB00DE11DE4
:105F2000F91F639FB00DE11DF91FBD01CF011124C1
:105F3000089597FB092E07260AD077FD04D086D056
:105F400006D000201AF4709561957F4F0895F6F7FA
:105F5000909581959F4F0895A1E21A2EAA1BBB1B15
:105F6000FD010DC0AA1FBB1FEE1FFF1FA217B30725
:105F7000E407F50720F0A21BB30BE40BF50B661F3B
:105F8000771F881F991F1A9469F7609570958095FF
:105F900090959B01AC01BD01CF01089597FB092E9F
:105FA00005260ED057FD04D0D7DF0AD0001C38F4E8
:105FB00050954095309521953F4F4F4F5F4F089535
:105FC000F6F790958095709561957F4F8F4F9F4F15
:105FD00008952F923F924F925F926F927F928F928D
:105FE0009F92AF92BF92CF92DF92EF92FF920F9368
:105FF0001F93CF93DF93CDB7DEB7CA1BDB0B0FB672
:10600000F894DEBF0FBECDBF09942A88398848882E
:106010005F846E847D848C849B84AA84B984C884C4
:10602000DF80EE80FD800C811B81AA81B981CE0FBB
:10603000D11D0FB6F894DEBF0FBECDBFED010895A0
:10604000EE0FFF1F0590F491E02D0994AA1BBB1BD6
:1060500051E107C0AA1FBB1FA617B70710F0A61B68
:10606000B70B881F991F5A95A9F780959095BC0189
:10607000CD010895911106C0803219F089508550E4
:0E608000D0F70895992788270895F894FFCF48
:10608E004E6F005965730054582074696D656F75B5
:10609E007421006D6F64756C65206C6F636B656445
:1060AE003F00486F70206368616E6E656C20002043
:1060BE0040200053004E2F4100386368002C002C06
:1060CE00205B005D20280029004E4F5420454E4194
:1060DE00424C45440053656E64696E672073657467
:1060EE0074696E677320746F2052580A005265737C
:1060FE00657474696E672073657474696E67732056
:10610E006F6E2052580A0041626F7274656420658A
:10611E00646974730A00696E76616C6964207365D4
:10612E006C656374696F6E000D0A496E76616C69F9
:10613E006420696E707574202D20646973636172BA
:10614E006465642107007363616E6E6572206D6F06
:10615E0064650053657474696E6773207361766548
:10616E006420746F20454550524F4D0A005265769B
:10617E0065727465642073657474696E67732066E6
:10618E00726F6D20454550524F4D0A004C6F616441
:10619E00656420666163746F7279206465666175EB
:1061AE006C74730A004B657920616E6420636861BC
:1061BE006E6E656C732072616E646F6D697A656464
:1061CE000A004F70656E4C52536E67205458207300
:1061DE0074617274696E672000206F6E20485720BC
:1061EE000050504D00525353490053444100534305
:1061FE004C00525844005458440041494E004C4201
:10620E004545500053504B54524D00534255530088
:10621E0053554D44004C4C494E440000342B340031
:10622E003800382B340031320031322B3400313605
:10623E000001000000C01200001A400AA1204EA565
:10624E00001B1E27522C23308025000005400AA17A
:10625E00204EA50020244EA52C2330004B00000616
:10626E00400AD0009D49007B289D492C233000E137
:10627E00000005400A4501D7DC03B81E0EBF0023FF
:10628E002E48E801008A400A6001555502AD1E20D5
:10629E00000023C88025000005400AA1204EA5005D
:1062AE0020244EA52C233000020002000200020022
:1062BE0002000200020002000200020002000200C0
:1062CE0002000200020002FF01610265026A026E14
:1062DE0002720276027A027E0284028B029002958C
:1062EE00029B029B029B029B0235019C02A002A212
:1062FE0002A602A902AE02350100070B0C10111501
:10630E0000160A1322312900000000E62E552B73C9
:08631E002EAD2E8D2ED62E00AF
:107E00000F92CDB7DEB7112484B714BE81FFF1D035
:107E100082E08093C00088E18093C10086E0809377
:107E2000C20080E18093C4008EE0CDD088249924E4
:107E3000CC24C394F5E0DF2EE1E1EE2E73E0F72EC3
:107E4000B6D0082F813479F4B2D08983C2D0898129
:107E5000823811F481E005C0813811F485E001C059
:107E600083E09ED09AC0823411F484E103C085344B
:107E700019F485E0B6D091C0853561F498D0082F0B
:107E800010E095D090E0982E8824802A912A880CC2
:107E9000991C82C0863521F484E0A3D080E0E1CF34
:107EA000843609F04CC083D082D0A82E80D0B82E62
:107EB00000E011E07CD0F80181938F01AE16D1F77C
:107EC00088D0FB2DF53489F4E0E0F1E00BC0F9999E
:107ED000FECF92BC81BC0894811C911C819180BD15
:107EE000FA9AF99AEA1598F358C08B2D863409F05E
:107EF00054C0F401F7BEE89507B600FCFDCFF401CD
:107F0000A0E0B1E02C9130E011968C91119790E0B7
:107F1000982F8827822B932B12960C01C7BEE895C9
:107F20001124329681E0A038B80761F7F401D7BE7A
:107F3000E89507B600FCFDCFE7BEE8952EC0843774
:107F4000F1F435D034D0182F32D0B82E42D0FB2DDA
:107F5000F63421F4F40105914F010CC0FB2DF534EA
:107F600049F4F999FECF92BC81BC0894811C911C04
:107F7000F89A00B5802F14D0115049F70EC08537FC
:107F800039F427D08EE10CD085E90AD08FE069CF93
:107F9000813511F488E017D01CD080E101D050CF9A
:107FA0009091C00095FFFCCF8093C600089580910A
:107FB000C00087FFFCCF8091C00084FD01C0A89560
:107FC0008091C6000895E0E6F0E098E19083808318
:107FD0000895EDDF803219F088E0F5DFFFCF84E10E
:107FE000DFCF1F93182FE3DF1150E9F7F2DF1F9166
:0E7FF0000895282E80E0E7DFEE27FF27099492
:027FFE0001057B
:0400000300007E007B
:00000001FF
